:020000000028D6
:104200000000010002000300040005000600070092
:10421000080009000A000B000C000D000E000F0042
:1042200010001100120013001400150016001700F2
:10423000180019001A001B001C001D001E001F00A2
:104240002000210022002300240025002600270052
:10425000280029002A002B002C002D002E002F0002
:1042600030003100320033003400350036003700B2
:10427000380039003A003B003C003D003E003F0062
:104280004000410042004300440045004600470012
:10429000480049004A004B004C004D004E004F00C2
:1042A0005000510052005300540055005600570072
:1042B000580059005A005B005C005D005E005F0022
:1042C00060006100620063006400650066006700D2
:1042D000680069006A006B006C006D006E006F0082
:1042E0007000710072007300740075007600770032
:1042F000780079007A007B007C007D007E007F00E2
:00000001FF
